:020000040000FA
:040000008301C5288B
:08000800FF00030E8301A000BC
:100010000A08A1000408A2008A010313831222081F
:10002000B4002308B5002408B6002508B700260848
:10003000B8002708B9002808BA002908BB002A0818
:10004000BC002B08BD002C08BE002D08BF002E08E8
:10005000C0002F08C1003008C2003108C3003208B8
:10006000C4003308C5008B18C6283408A200350820
:10007000A3003608A4003708A5003808A6003908F0
:10008000A7003A08A8003B08A9003C08AA003D08C0
:10009000AB003E08AC003F08AD004008AE00410890
:1000A000AF004208B0004308B1004408B200450860
:1000B000B3002208840021088A00200E8300FF0E6E
:1000C0007F0E09002E08AC070318AF0A2F08AD07F2
:1000D00000342F08A3002E08A400A501A6011030AB
:1000E000AB00A40DA30DA60DA50D24102C08A8008F
:1000F0002D08A7002608A9002508AA002808A6029E
:100100000318852803198528A70A2708A5020318BC
:100110009E2803199E282908A6002A08A500A40DD8
:10012000A30DA60DA50D2410AB0B76280310A50C6E
:10013000A60C2308AD002408AC000034A40DA30DC8
:10014000A60DA50D2414AB0B76280310A50CA60C48
:100150002308AD002408AC0000342C08300203183A
:10016000B6280319B6280130B0000034B0010034BD
:100170002F082D02031DC3282E082C02031DC3289F
:100180000130B0000034B0010034CE2803138312D4
:100190000130C8070318C70A8B10352803138312D0
:1001A00000308316850001308600FE308312860001
:1001B0001F308500C801C701C601831601170B1740
:1001C0000B168B170B1783129101FF3083169200C9
:1001D00000308312950097010F3097040030970488
:1001E000831686118312121583168C102130831208
:1001F000AE00F830AD00B930AC00AC0BFD28AD0B53
:10020000FB28AE0BF9284430B100B10B05290000E2
:100210000000031383121030AE007330AD00CE30F7
:10022000AC00AC0B1129AD0B0F29AE0B0D2913300F
:10023000B100B10B19290000000000008B130B1353
:100240004808AC004708AD002C08B2002D08B300E8
:100250000230AC000030AD003308AF003208AE0011
:100260006920031383122C08CA002D08C900CA187C
:100270003B2986103E29031383128614031383122D
:100280004A1944290611472903138312061503133B
:1002900083124A1A4D290612502903138312061697
:1002A00003138312CA1A562986125929031383127B
:1002B0008616031383124A1B5F2906136229031350
:1002C0008312061703138312CA1B682986136B292E
:1002D000031383128617031383124A080939850012
:1002E0004808AC004708AD002C08B2002D08B30048
:1002F0000030AC000130AD003308AF003208AE0072
:100300006220031383122C08C8002D08C700470879
:100310000339C70003394708AD004808AC002C1862
:1003200017161712AC1897169712AD0CAC0CAD0C33
:10033000AC0C2C089500C8014814C70103138312A4
:060340008B170B170929C1
:00000001FF
